:030000000219FDE5
:03000B000200AA46
:03002B0002015F70
:03005B000202F5A9
:030073000202DBAB
:1000800002030406080C10182030406080040608A3
:100090000C10182030406080A0C000070F1F3F0DDB
:1000A0000D0403060D0502030202C2AFC0D0C0E07A
:1000B000206217E5256002E473E525F4F58A758B67
:1000C00000D262D0E0D0D0D2AF3285268AC262E5BB
:1000D00026F4602F758B00D0E0D0D0C293C295C2B9
:1000E00097D2AF32C293C295C297206E0C20660998
:1000F000740ED5E0FDE57E4290758B00D0E0D0D047
:10010000D2AF32758A00C28DD26201F901B930686E
:1001100005206602D29301B9306805206602D295A7
:1001200001B9306805206602D29701B9C2923068E1
:100130000A206607740CD5E0FDD29301B9C2943051
:10014000680A206607740CD5E0FDD29501B9C29605
:1001500030680A206607740CD5E0FDD29701B9C259
:10016000AFC2AD53E6EFC0D0C0E0D2D3D2AFC2CE63
:10017000E52A6007207449152A21C07800790020FB
:10018000742EE580307E01F430E30278FF53DACF3D
:10019000207E0343DA20307E0343DA10C2D8C271D6
:1001A000E580307E01F430E30279FFC3E89970CB3B
:1001B000306103752A40207403752A40885FD2702D
:1001C00020740DE52B6004152B21D043DA01C2D831
:1001D00020700221E3A85F206102C2702074022116
:1001E000E188227882B60403852224C3E525944061
:1001F0004002D26420CF0AD0E0D0D043E610D2AD86
:1002000032C2CF053A7802E52A6005307402152A19
:10021000C3E55F94014005756200412D756300756B
:100220006C00E5622401F56250037562FF7982B7C4
:10023000020D306D1DC3E52294324016854D2279A2
:1002400082B7030E306D0BC3E52294324004798EE1
:100250008722C3E5239522600840041523416105E8
:1002600023D8CA056CE56C7002156CD56D63756D8D
:10027000017805C3E56C956E4057C3E56C956F50EA
:10028000087801756D03020295C3E56C9570500501
:100290007801756D01C3E5659524401E7982B70428
:1002A0000241C6206D14852465E56C046003856EEB
:1002B0006C756D0175233C0202D1E565285005750A
:1002C00065FF41C6F565E5650470067563FF756CED
:1002D000FFD0E0D0D043E610D2AD32C2AFC0D05391
:1002E000E67FC26075910085569485579575910497
:1002F000D0D0D2AF32C2AF53E6EFC2ADC0D0C0E073
:10030000C0F0D2D3D2AFA8FBA9FCC2D83071026131
:100310005C53DACF207E0343DA10307E0343DA20C9
:10032000D271E580307E01F420E3026133882789B1
:1003300028A14153DACF207E0343DA20307E0343E5
:10034000DA10C2D8C271307402A12D7800E5803075
:100350007E01F430E302A12D885FA11553DACF208E
:100360007E0343DA20307E0343DA10C2712061023B
:10037000813553DACF207E0343DA10307E0343DA2F
:1003800020C2D8D271885A895BC3E89558F8E9959C
:1003900059F97B007E087A00C3E8948CE9940050F8
:1003A00005755E008127882178A2E6A8216055C3E3
:1003B000E894C8E994005008E4D2E4FB7A0A810288
:1003C000C3E89468E994015008E4D2E3FB7A0F8112
:1003D00002C3E894D0E994025008E4D2E2FB7A1E0A
:1003E0008102C3E894A0E994055008E4D2E1FB7AC5
:1003F0003C8102C3E89498E994085008E4D2E0FBF9
:100400007A787E00C3E8955CFCE9955DFD30E70AEB
:10041000ECF42401FCEDF43400FD755E00C3EC9AAD
:10042000ED9E5003755E01885C895D855A58855B39
:10043000597802A115C3E89527F8E99528F9307C89
:100440000281F9307B0281F9307A0281F220750253
:100450008158E9FDE8FC8177E9C313F9E813F83026
:10046000790281F2E9C313F9E813F830780281F2D6
:0F047000E9C313FDE813FC20612CC3EC941CEDD1
:10047F0094024002818EED701EC3EC94C850180593
:10048F0029E52970021529C3E529940A5002A12DE7
:10049F00755F00D270A12DE5296002152974002027
:1004AF007F037896E624FAFEE43400FFC3EC9EFC4B
:1004BF00ED9FFD50067800790081F9C3EC94FFEDB4
:1004CF009400400678FF790081F9EC8575F0A4C59A
:1004DF00F0A2F733F87900400302051578FF790091
:1004EF00020515E9C313F9E813F8307C0EE9600231
:1004FF0078FFC3E81338F8E43400F9C3E894FFE950
:10050F009400400278FF885FD270206102A12D74A1
:10051F001FF4552F4BF52FC274EB7002D274752A4E
:10052F0040307403752A0A306102A14120740353CD
:10053F00DAFE207403752B20D0F0D0E0D0D0D2ADEE
:10054F0043E6103279010205717903020571790AC8
:10055F00020571791E020571796402057179C8026D
:10056F0005717817E4D5E0FDD8FAD9F6227A147B15
:10057F00780205987A107B8C0205987A0D7BB4026D
:10058F0005987A0B7BC80205987902B27DE4C29474
:10059F00D5E0FDD295D5E0FDC295D5E0FDD294D53D
:1005AF00E0FDD293E576D5E0FDC2937496D5E0FDDC
:1005BF00D9D9EAF8D5E0FDD8FBDBCEC29422C37CB3
:1005CF00007D0075F00005F0EA33FAEB33FB50F6CF
:1005DF00EB13FBEA13FAC3E9FFE8FEE89AF8E99B8D
:1005EF00F95004EFF9EEF8B3EC33FCED33FDD5F031
:1005FF00DFEDF9ECF822E889F08A20D2D4F8A9F0DF
:10060F007B0030F70B7BFFF42401F8E9F43400F999
:10061F00E88520F0A4ADF0F8E98520F0A4AFF0FE56
:10062F00ED2EF974003FFA7C04C3EA13FAE913F9CB
:10063F00E813F8DCF48BF030F70AE8F42401F8E95A
:10064F00F43400F9E889F0C2D4F8A9F0227882B620
:10065F0004030206FBC3E55F9419401EE52D540603
:10066F007018206D3678057994E7146007780A14AE
:10067F0060027812C3E54198401F306D09856765A8
:10068F00756CFF756D01852224E4F545F546F54738
:10069F00F548F549C26D0206FBD26D7994E71470E7
:1006AF0013E523F43333F913F8E9540104F9E8544B
:1006BF00FE0206EFE714147014E523F4333333F915
:1006CF0013F8E9540304F9E854FC0206F7E523F4A0
:1006DF0033333333F913F8E954070404F9E854F8C2
:1006EF00C39440F8E99400F98845894622C3E5414F
:1006FF0013F9E54013F8C3E54598F8E54699F95025
:10070F000CC3E89480E994FF4016020733C3E894C2
:10071F007FE994005003020733787F790002073393
:10072F00788079FF884A894B22E54A2547F8E54BBF
:10073F003548F9854B20E4300701F43549FA30E7A5
:10074F0009C3EA94F04015020771C3EA940F5003EE
:10075F0002077178FF79FF7A0F020771780079002D
:10076F007AF0C3E5249564500AC374019524500BA5
:10077F0002078FE54B20E70E02078FE54B30E706A8
:10078F00884789488A492278A4E6FAC3E54A33F8AC
:10079F00E54B33F9D105E930E70BC3E89480E994D1
:1007AF00FF4013E1C9C3E8947FE994005002E1C907
:1007BF00787F7900E1C9788079FFE820E715C3E5F4
:1007CF002398F84009C3E8940140030207F0780129
:1007DF000207F0E8F424012523F840030207F0781C
:1007EF00FF884C2278A5E6FAA848A949D105E93037
:1007FF00E70CC3E89401E994FF4016020824C3E80C
:10080F0094FFE99400500302082478FF790002084E
:10081F0024780179FFE920E715C3E54C98F84009E2
:10082F00C3E89401400302084B780102084BE8F437
:10083F002401254CF8400302084B78FF88242278C6
:10084F00FFC26420693D206A12D264C3E541940A55
:10085F004009C3E52594405002C26479A1E76023A3
:0D086F00E541601F74FF8541F0848539F07C
:10087C00306A0375F005A4F8C5F0600278FFC3E890
:10088C0095675002A867886622C3E5409440E5410D
:10089C009401E56650031401A6046002F566227803
:1008AC0083E6F520120F5F75E89012055375E890FA
:1008BC00E5E820ECFBA8BDA9BE120FF975713075E7
:1008CC007200C3740013FD7430606613FC74302C1A
:1008DC00FC74003DFDECFAEDFBC3E89AE99B401477
:1008EC00E5712430F571E5723400F572EA2CFAEBFF
:1008FC003DFB80E5AE71AF72C3E57213F9E5711380
:10090C00F8C3E913F9E813F87A03C3E913F9E81308
:10091C00F8DAF7AA201A70097571007572000209CD
:10092C003D1AEA6008EE28FEEF39FFDAF88E718F77
:10093C00722275E890227883E6FFE5E820ECF7A8B0
:10094C00BDA9BE0573C3E57394084052757300E9E5
:10095C00FA79A0E76044EA7007E574601B02097835
:10096C00C3E895746010E5745006600C1402098499
:10097C000460F9020984E574F574C394A8401B75EE
:10098C0064C0C394054013756480C39405400B7513
:10099C006440C39405400375640075BB0122EFC32A
:1009AC009401601F7430601BC3E894FFE9940350FA
:1009BC0012C3E89571E995725009E564600C1564F1
:1009CC000209D6E564F460020564A864C3E52498C2
:1009DC005002A824C3E89565400AA865E565F46053
:1009EC000385656488258826E573B4070375BB1EEB
:1009FC0022743279A687F0A4C5F0A2F733F8C3E8C5
:100A0C0095644002A86488228824882588268867F3
:100A1C00227540007541F022C2AF75C820A8CCA940
:100A2C00CDAA3A30CF010A75C824D2AFAB3BAC3C4F
:100A3C00883B893CC3E89BF8E99C206908F930673E
:100A4C000261394196AD3D8A3DF9EA9DFA60047820
:100A5C00FF79FFAE3EAF3F8B3E8C3FC3EC9FFCC398
:100A6C00E99CF542A83BA93CC3E89EF8E99FF9C371
:100A7C00E54113FBE54013FAE82AF540E93BF54163
:100A8C0050067540FF7541FF41E0AA40AB41AC40B8
:100A9C00AD417E047F02C3EB940440021E1FC3EBE6
:100AAC00940840021E1FC3ED13FDEC13FCDEF7C3CC
:100ABC00EA9CFAEB9DFBEF6009C3E913F9E813F824
:100ACC00DFF7EA28FAEB39FB8A408B4150067BFFB3
:100ADC008B408B41C3EB94025002D2673069047F88
:100AEC0003610B7892E6FFC3E537948240110FC384
:100AFC00E53794A040010FC3EF940640027F057EBA
:100B0C0006E541C4540FF9E541C454F0F8E540C47E
:100B1C00540F28F8C3E89EFAE99400FB4009C3EA95
:100B2C009402EB940050047A02E4FB6185AA40AB7A
:100B3C0041EBC4FEEAC4540F4EFCC3EA9CFAEB949E
:100B4C0000FBC3E813C313F8EA28FAEB3400FB8A62
:100B5C00408B41C3EB94024002C2677806EBC4FEA3
:100B6C007B00EAC4540F4EFAC3EA98FA4005C394CA
:100B7C000250027A027892E6FF306002618585525B
:100B8C0056855357D26043E680C3E49AF8E49BF948
:100B9C00306702811FE8FAE9FBD3E913FDE813FC87
:100BAC0088528953C3EF94036038EF20E00DE82C92
:100BBC00F8E93DF9ECFAEDFB020BDAE828F8E93933
:100BCC00F9C3E82402F8E93400F97AFE7BFFC3EF9D
:100BDC009403400E8A548B55884E894F8C508D51FE
:100BEC008153885489558A4E8B4F8C508D51306966
:100BFC0020C3E53394034019E542A2E713F8E55509
:100C0C00F4240138400B20E7087554FFF42401F557
:100C1C00558153E8FAD3E813FC8852C3EF94036070
:100C2C0020EF20E007E82CF8ECFA813FE8282402BA
:100C3C00F87AFEC3EF940340088A54884E8C508196
:100C4C005388548A4E8C50E56BC3335002646BF559
:100C5C006B306002815D753402D26043E680E52D15
:0F0C6C0054066026A840A941C3E913F9E813F81C
:100C7B00C2AF53E67F759100C3E498F594E499F500
:100C8B0095759104D26043E680D2AF22D26575444C
:100C9B0000752000306B03752040020CB6D26575D1
:100CAB004400752040306B03752000D2AF780120D3
:100CBB006722E52D54066002C265C3E541940540E9
:100CCB0013780294054008780394054002780630A7
:100CDB006902780A206019E544601530690AC3E59A
:100CEB003394034003D53406D2AFD26CA1909165F7
:100CFB00D2AF0000C2AF206726E541C3FB940F4083
:100D0B00027B0FEB240530730123306A0274282019
:100D1B00620123F93069027982E58BC39940B505ED
:100D2B0044E59E7005E59B020D37E59A5440B520CE
:100D3B0002A17A30690A08C3E8940A40010881DFEE
:100D4B0020650281B6C26553E67F7591003067104E
:100D5B007594007595FE759104D26043E68081B65B
:100D6B00AE40AF41C3E49EF594E49FF595A161C3FA
:100D7B00E5339402500281B630650281B6D802A1E8
:100D8B008E81DFC26C53E67F759100855494855537
:100D9B0095759104854E56854F57D26043E680D2A8
:100DAB00AFE52D54066008206A020533020DCA30E8
:100DBB006C0D206B0A2065071581158102164322E5
:100DCB0078003064053065027801E53775F007A4CB
:100DDB00F9E5F028F5F0E9A2F013A2F113A2F21352
:100DEB00F537C394785003753778C3E5379538409A
:100DFB0008D266C293C295C297306002C104855077
:100E0B0056855157D26043E68022207D14C2AF75C0
:100E1B004302C294D292D2AF759F33759E00020FDC
:100E2B00F6C2AF754302C294D296D2AF759F33759B
:100E3B009E00020FF6307243207D20C2AF75430334
:100E4B0090013D757E10C297C296306204D295C157
:100E5B005ED294D2AF759E23020FF6C2AF754303D9
:100E6B0090013D757E10C293C292306204D295C13F
:100E7B007ED294D2AF759E22020FF6207D17C2AFA1
:100E8B00754303900118C297306202D295D2AF75A9
:100E9B009E23020FF6C2AF754303900118C2933025
:100EAB006202D295D2AF759E22020FF6207D11C23F
:100EBB00AF754304C292D296D2AF759E22020FF643
:100ECB00C2AF754304C296D292D2AF759E23020F66
:100EDB00F6307249207D23C2AF75430590012C7506
:100EEB007E04C295C294306204D293C1FAD292D2DC
:100EFB00AF759F33759E00020FF6C2AF7543059019
:100F0B00014E757E40C295C294306204D297E11DAA
:100F1B00D296D2AF759F33759E00020FF6207D1AC5
:100F2B00C2AF75430590010EC295306202D293D2C7
:100F3B00AF759F33759E00020FF6C2AF75430590D8
:100F4B000122C2953062E8D297D2AF759F33759E5E
:100F5B0000020FF6207D11C2AF754306C296D294E4
:100F6B00D2AF759E23020FF6C2AF754306C292D263
:100F7B0094D2AF759E22020FF6307242207D20C2B2
:100F8B00AF75430190014E757E40C293C2923062A1
:100F9B0004D297E1A2D296D2AF759E22020FF6C26F
:100FAB00AF75430190012C757E04C297C2963062D7
:100FBB0004D293E1C2D292D2AF759E23E1F6207D8B
:100FCB0016C2AF754301900122C293306202D297D1
:100FDB00D2AF759E22E1F6C2AF75430190010EC2EE
:100FEB0097306202D293D2AF759E23C266229001D4
:100FFB000C757E00C293C295C297C292C294C296E0
:10100B00C262227880760708760708760108760494
:10101B000876FF0876FF087607087602087601083F
:10102B007601788C76010876000876B40876FF088E
:10103B0076FF0876FF0876030876FF0876010876B8
:10104B00FF0876250876D00876780876C8087604E7
:10105B000876FF08760108760008767A087610087D
:0F106B0076010876010876000876FF227887E67E
:10107A00FFC2727888C27DE630E102D27DC27E78F4
:10108A0089E630E102D27EC3EF94026008758E01D0
:10109A00D2730210A4758E00C273227880E614906F
:1010AA0000809378A4F67881E6149000809378A55E
:1010BA00F67886E61490008D9378A6F6789FE6F87F
:1010CA00700108C3E8941140027811E82828F56EE7
:1010DA00256E256E28F56F256E2828F570789CE612
:1010EA007538FF75390CB402067538A075390AB41B
:1010FA00030675388275390578A3E61490009A9329
:10110A00F569120FF922227896E6FA7897E6FB78C3
:10111A0088E6B40305C3EB940EFB307F047A007BA8
:10112A00FFC3EB9AFCC3948250027C82757500055A
:10113A0075EC8575F0A4C3E5F0947D40F222D27F68
:10114A0031111205627A007B007C10120558E55FA6
:10115A002AFA74003BFBDCF37C04C3EB13FBEA13AF
:10116A00FADCF7FEC27F311122E5EF20E603752093
:10117A00000520903DFFE520146006901FFF1460D3
:10118A00009304600375EF1253D9BF7581C043FF02
:10119A008012055375EF0243B203E5B3240420E736
:1011AA000DF521E5B120E0068521B343B101120F07
:1011BA00F97580FF75A40075F1FE75D4F775900274
:1011CA0075A5FC75F2FC75D50075A0FD75A60275AE
:1011DA00F30275D60075B0FF75A70175F4FF75E2C5
:1011EA0041E4F8F6D8FD756B01110E12168B78984A
:1011FA008676753001C2AF12056C12057C12056243
:10120A0012058312056212058A1205621217AD12BF
:10121A00056C12056C120567C2AF78FA79FA308349
:10122A0007D9FBD8F7021C00117711A5311031112B
:10123A0078988676120FF975885075891275C824C0
:10124A0075910475D84075A82275B80275E690752F
:10125A009B80759D00759A80759C0075D10E75BC32
:10126A005875BB0175BA1F75E880120553D2AF12C3
:10127A0008AB53DACF207E0343DA20307E0343DA09
:10128A001043DA01C2D8C27112056CD2617B037AAB
:10129A000CE55E70077A0CDB03021222120562204B
:1012AA007003021222C270E55FC3940240E1E52F87
:1012BA00541F856160F561B560D5DAD5C26153DA2C
:1012CA00CF207E0343DA20307E0343DA10C2D8C22D
:1012DA007178A2E67008D274E52F54E0F52FC27532
:1012EA00752900120567307409C3E529940A40027A
:1012FA00D27512055878023074027800C3E55F98F7
:10130A0040F0C2AF12057C12057C12057CD2AF12E6
:10131A00056C754D00120558788CE6C3940150038C
:10132A000213F5E530C3940150030213F520743516
:10133A00C3E55F94FF50030213F5C2AF120591D2C1
:10134A00AF120567C3E55F940150EFC2AF12057C87
:10135A0012055D12057CD2AF120567C3E55F94FFE3
:10136A0040E90218327F05D27F3111120567C2AFF8
:10137A00C27F3111AE5FC3E55F947FD2AF40761270
:10138A000553C2AF120591D2AFDFDC3148C3EE94E8
:10139A00057897F612056C1216CC1217B57F0AD289
:1013AA007F3111120567C2AFC27F3111AE5FC3E54B
:1013BA005F947FD2AF50E6120553C2AF12057C127A
:1013CA00055D12057CD2AFDFD63148EE240578964A
:1013DA00F612056C1216CC1217E41205673111C306
:1013EA00E55F94FF50026137021832C3E55F954DFD
:1013FA004003855F4D12056778017988E7B40302D7
:10140A007805C3E55F984002611FC2AF12059112C9
:10141A000591120591D2AF12056C753000E4F531D1
:10142A00F5320531E531F470390532789AE67819E2
:10143A00146012783214600D787D14600878FA14FA
:10144A006003753200C3E53298401715327531B41E
:10145A0078998676C2AF120591D2AF7898867612BD
:0E146A00056712055DE52A7005307402412207
:1014780078012074027806C3E55F9840A7120567D3
:10148800E52A7003021222C2AF120FF9E4F522F521
:1014980023F524F525F526F56AD2AF7885E6C3331A
:1014A800F568E4F545F546F547F548F549F573F56A
:1014B8002CF52DF53775730875BB1E1205531209E7
:1014C8003EE5E820ECFBA8BDA9BEE97001F88874E8
:1014D80012094275730875BB1E7887E6FE760211FD
:1014E800777887EEF6C2AF7564FF1209FD8522642E
:1014F800852265852266D2AF75220175240175257E
:101508000175260185636C756D017888E6B403075B
:10151800C27D307602D27DD268D269753300120F4F
:101528005F120F84120A1D120A24120A1D120A24BD
:10153800120A1D02154AC2AF1177D2AF7573007532
:10154800BB01120CA812065C120DCB120E15120A62
:1015580024120C97306D031206FC20670312084E04
:10156800306703120895120DCB120E40120A24128E
:101578000CA8306D03120738120DCB120EB7120AE1
:1015880024120C97306D03120796120DCB120EDC45
:10159800120A24120CA8306D031207F3120DCB1295
:1015A8000F5F120A2412093E120C97120DCB120F6C
:1015B80084120942120A2430692F206B2C85676433
:1015C80085676585636C756D0179187A0CC3E53399
:1015D800994009C269D26A8A350215F1C3E55F9458
:1015E80001400302154A02164B306A1B206B18E5AE
:1015F80035147004C26AA13EF535C3E55F94014015
:101608000302154A02164B753600C3E56294014081
:101618000985676585636C756D01C3E56278FA981D
:101628005021307404E52A601A78F0306B0585671C
:10163800647820C3E541985002A14A0536E55F6009
:1016480002C14E753600C2AF120FF97887E6FE76F2
:101658000211777887EEF6E4F522F523F524F525CF
:10166800F526F568C268D2AF120553120FF9307427
:1016780006E52A70024122788DE6C39401400241B2
:10168800FC8127901A0D782012170EE520B4A50CBE
:10169800A312170EE520B45A030216AC110E121647
:1016A800CC0216CB901A0378807B0A12170EA30877
:1016B800DBF9901A0F788C7B1812170EA308DBF948
:1016C800901A2722C2AF12174D121727901A0074CA
:1016D8000E121713A37404121713A37414121713FA
:1016E800901A0378807B0A121712A308DBF9901A64
:1016F8000F788C7B18121712A308DBF912176012E7
:10170800173E901A2722E493F622E6438F01538F5F
:10171800FD75EF0275B7A575B7F1F0538FFE22433B
:101728008F02438F0175EF0275B7A575B7F1901A4F
:101738000DF0538FFC22901A0D74A5F113901A0E18
:10174800745AF113227A3079D07820901A40F10E29
:10175800E520F709A3DAF7227A3079D0901A40E722
:10176800F11309A3DAF922AB77A878BB01027980D3
:10177800BB02027981BB03027982BB04027994BB64
:1017880005027983BB06027986BB07027992BB08FA
:10179800027987BB0902799CBB0A027988BB0B02D4
:1017A8007989E8F7227C0512056CDCFB22C2AF12AE
:1017B800057C12058312058A12059112055D120532
:1017C8007C12058312058A12059112055D12057CAB
:1017D80012058312058A120591D2AF22C2AF1205F3
:1017E8009112058A12058312057C12055D12059176
:1017F80012058A12058312057C12055D12059112E5
:10180800058A12058312057CD2AF22AE77AF78C263
:10181800AF12057C12057C12057C12055DDEF21202
:10182800059112055DDFF8D2AF221217B51217AD78
:101838001217AD75770175780175790011137C055C
:10184800AD5F12056CC3ED955F70F5C3E55F94015C
:10185800400AC3E55F94FF403702187512176F12EC
:0F18680016CC1217B5C2AF75EF121217ADDCD147
:101877000579C3E5799403500280C21217AD057844
:10188700E5771490009F93F808C3E5789850028095
:10189700A91217AD1217AD0577C3E577940C50025F
:1018A700809512100E1216CCC2AF75EF121217AD3B
:0319FD0002117361
:101A00000E041407070104FFFF07020101A55A0194
:101A100000B4FFFFFF03FF01FF25D078C804FF01DA
:081A200000FF10010100FFFFAF
:101A4000235467794B4631323041485623202020B9
:101A500023424C48454C4923463331302320202033
:101A60002020202020202020202020202020202076
:101C0000C2AFC2D353D9BF7581C043B20343FF8073
:101C1000752438752503B1C975EF0275E24043F1AB
:101C20000853A4F775D400D2837DFA780379E67C53
:101C300010752200752300901DD67B0675249875BB
:101C400025013083028142208308D8FBD9F9DCF7D3
:101C500081B4308308D8FBD9F9DCF781B4B189E4C9
:101C600093A3C39A6004DDC381B4DBDBB17B600264
:101C7000812B7B08E493FAA3B15CDBF87A30B15C8A
:101C8000752200752300B17BEAFCEBFDC3ED94FEE9
:101C9000400EB17B8A278B28ED30E0048A828B834B
:101CA000B17B7AC270D8C3ED94FE601350CEBD00F4
:101CB00025EC60097520007521FF0200008100A855
:101CC00027A9280809D804D90281D3B17FEA89AAB3
:101CD000F281C50D81A0C3ED94035049EDA2E092BD
:101CE000007AC5C3E5829400E583941C50902000DF
:101CF00010438F02438F0175B7A575B7F1F030001F
:101D00001FA827A9280809438F01538FFDD804D99C
:101D100002A12089AAE275B7A575B7F1F0A3A10DBC
:101D2000538FFC817C7AC1BD030CE493A3FAB140CC
:101D3000DCF8B138817C817EAA22AB23B15CEBFA5E
:101D4000EA6222752608C3E52313F523E52213F57D
:101D50002250066323A0632201D526EAB1C9B1C986
:101D600075260AEAF4200102D283300102C283B14F
:101D7000C9C3134002C201D526EB22B17FEAFB2082
:101D80008302A17F308302A184752608AE24AF258B
:101D9000C3EF13FFEE13FEB1CDB1C9C3EA13308315
:101DA000024480FA30E703632201C3E52313F523DD
:101DB000E52213F52250066323A0632201D526D91C
:101DC000E52265236523F52222AE24AF250E0FDE22
:101DD000FEDFFCD20122424C48656C693437316326
:041DE000F3100601F5
:00000001FF
